:020000040000FA
:0400000086EF02F095
:08000800F76A180FF66E000EF6
:10001000F7220900F55012004F4B0A0D0000F76A55
:100020002E0FF66E000EF7220900F5501200256C17
:10003000750A0D4D4158313434204348303A20255B
:100040006C752C2025662C20256C750A0D00F76A2E
:100050005E0FF66E000EF7220900F55012004D41BA
:1000600058313434204348313A20256C752C2025F2
:10007000662C20256C750A0D0000F76A8A0FF66E53
:10008000000EF7220900F55012004144433A2025A2
:100090006C752C2025662C20256C750A0D0A0D0028
:1000A000040EEA6E120EE96EEF500EE00F0E016EB6
:1000B000006A002EFED7012EFBD78F0E006E002E99
:1000C000FED70000EF2EF2D7000C8E0E006E12C489
:1000D00001F011C402F0036A015209E102C001F00B
:1000E000026A080E005E015202E1006A08D0D89050
:1000F00001BE04D0023601360006F9D7019E000089
:10010000000C04011F51D8B471D0006E2351D8B433
:100110006DD0002604E3810E002668E204D07F0E35
:10012000005E64E363E020C427F42451271B208F82
:10013000248F22512603F4CF29F421512503F4CF33
:1001400003F0F3CF28F42603F3502927F450282393
:10015000000E032222512503F3502927F4502823AF
:10016000000E026A0322022220512603F3502827A0
:10017000F4500322000E022220512503F3500326DF
:10018000F4500222000E016A012222512403F3508E
:100190002827F4500322000E0222012221512403B9
:1001A000F3500326F4500222000E012220512403B2
:1001B000F3500226F4500122002A01BE05D0283750
:1001C0000336023601360006000E28AF0AD0032A95
:1001D00002220122015005E1025003E1035001E136
:1001E000002A27BF018E27AF019E04D0006A016A52
:1001F000026A036A00000001000CEACF1AF4E9CF9A
:1002000019F404011339F009156F1527E20F166F61
:10021000320F186F13510F0B162716271827E90FE7
:10022000176F1727172712390F0B1727182717379C
:100230001837181F183712510F0B18271537070ECC
:10024000146F0A0E17071827FDE316071727FDE39B
:1002500015071627FDE314071527FDE3040EEA6EC4
:10026000140EE96E070E1915199DE926180EE95CA2
:10027000D8B4198DEF50006E08E119BD06D019B938
:100280000CD019B702D0200E03D019871999300E5F
:10029000002600509EA8FED7AD6EEE5019ADE6D7F1
:1002A0000001000C04011F51B6081F6F036A20C42F
:1002B00023F4208FD89020332133223303320232AB
:1002C000013200321F2FF6D723AF0BD0001E011EC4
:1002D000021E031E002AD8B4012AD8B4022AD8B4B8
:1002E000032A0001E0EF01F0006A016A026A036A72
:1002F0000401276B286B296B2A6B265125112411C9
:1003000023112CE0200E2B6FD8901F372037213778
:1003100022372737283729372A3726512A5D08E11F
:100320002551295D05E12451285D02E12351275D16
:100330000FE32351275F2451D8A0243D285F255186
:10034000D8A0253D295F2651D8A0263D2A5FD88018
:1003500000360136023603362B2FD6D70000040EA6
:10036000EA6E270EE96E0001000CE9500401176FD8
:100370001651196F1BE015C422F414C421F413C4E0
:1003800020F412C41FF4266B256B200E246F820EFE
:10039000236F0001B6DE03C015F402C014F401C0DF
:1003A00013F400C012F40401192FE5D715C422F488
:1003B00014C421F413C420F412C41FF4000172D732
:1003C00003C015F402C014F401C013F400C012F409
:1003D000040115AF0DD01707178B121F131F141F21
:1003E000151F122BD8B4132BD8B4142BD8B4152B3B
:1003F0003B0E1E6F9A0E1D6FCA0E1C6F1B6B0A0EF2
:10040000196F1651D8B4172B15C422F414C421F453
:1004100013C420F412C41FF41EC426F41DC425F412
:100420001CC424F41BC423F400015EDF0150EFCF91
:1004300012F4ECCF13F4ECCF14F4ECCF15F400521B
:1004400013E104011629195DD8A402D000010CD0D3
:1004500017510DE00F0B195D01E03CE217BF3AD0D8
:1004600017BD05D0200E31D0200E0401171717AB91
:100470000DD0179B1651D8A417070050176F2D0EDB
:100480009EA8FED7AD6E1751006E176B1651195D01
:100490000BE10050176F2E0E9EA8FED7AD6E1751C0
:1004A000006E200E1717000E300E17AB0ED0179BE4
:1004B0001651D8A417070050176F2D0E9EA8FED70F
:1004C000AD6E1751006E176B300E002600509EA8BF
:1004D000FED7AD6E1EC422F41DC421F41CC420F44A
:1004E0001BC41FF4266B256B246B0A0E236F0001BF
:1004F000FBDE03C01EF402C01DF401C01CF400C0EA
:100500001BF40401192F80D70001000CF86AD09E5B
:10051000EA6AE96AB896190EAF6E260EAC6E900EB6
:10052000AB6EC150C00B0F09C16E070EB46E056AE9
:10053000C150C00B0E09C16EC090C082C084C08E75
:10054000C280880ED56ECD6A000ECA6E7F0ECB6E4D
:10055000B150480B8509B16EB70EB1169484BD6ACF
:10056000BD6AB1169482BA6ABA6AC69A949E93809A
:100570009392210EC66E000EC76E93948A84939256
:100580008A92016EC250C30B0110C26E010E0401AB
:10059000126F000185DD0C6A0B6A020E0401116FF7
:1005A000FA0E126F00017CDD0401112FF9D7116BD7
:1005B0001151000129DD0401112B006E00509EA88D
:1005C000FED7AD6E040E115DF3E1C80E126F00018F
:1005D00067DDB36AB26A0401116B93948A949380C5
:1005E00081A0FDD7C950C96AC7A0FED7C9CF14F4EE
:1005F000C950C96AC7A0FED714C413F4C9CF12F4F6
:10060000000E13B9010E115D16E093948A84000068
:1006100093948A94938081A0FDD7C950C96AC7A0DA
:10062000FED7C9CF14F4C950C96AC7A0FED714C4F5
:1006300013F4C9CF12F493948A841235146F1335CE
:10064000156F143715371437153714371537F00E63
:1006500014171531136F1431126F13331233133310
:100660001233133312330F0E131712C401F013C4D5
:1006700002F002C008F001C007F0D8900B34026EFF
:100680000C34036E0250110FE96E000E0320EA6E67
:1006900008C0ECFFED5207C0EFFFB250B3CF03F03C
:1006A000096E03C00AF0106A0F6A200E0E6E750EF6
:1006B0000D6E08C012F407C011F4000106DD03C07E
:1006C00022F402C021F401C020F400C01FF410C0C5
:1006D00026F40FC025F40EC024F40DC023F411DD60
:1006E00003C010F002C00FF001C00EF000C00DF00A
:1006F000100EE96E0CC013F40BC012F47EDD030E75
:100700000401116F115100018ADC0401112B006EEC
:1007100000509EA8FED7AD6E110E115DF3E1100ED4
:10072000E96E08C013F407C012F4000166DD2C0E58
:100730009EA8FED7AD6E200E9EA8FED7AD6E890E88
:10074000E96E10C015F40FC014F40EC013F40DC000
:1007500012F4060E0401166F000107DE2C0E9EA88F
:10076000FED7AD6E200E9EA8FED7AD6E100EE96EC0
:100770000AC013F409C012F440DD0A0E9EA8FED789
:10078000AD6E0D0E9EA8FED7AD6EB36AB26A010EB5
:100790000401116F93948A94938081A0FDD7C9506E
:1007A000C96AC7A0FED7C9CF14F4C950C96AC7A087
:1007B000FED714C413F4C9CF12F4000E13B9010EFE
:1007C000115D16E093948A84000093948A94938038
:1007D00081A0FDD7C950C96AC7A0FED7C9CF14F4FC
:1007E000C950C96AC7A0FED714C413F4C9CF12F404
:1007F00093948A841235146F1335156F1437153797
:100800001437153714371537F00E14171531136FC9
:100810001431126F13331233133312331333123371
:100820000F0E131712C401F013C402F002C008F037
:1008300001C007F0D8900B34026E0C34036E0250E6
:10084000110FE96E000E0320EA6E08C0ECFFED52B6
:1008500007C0EFFFB250B3CF03F0096E03C00AF038
:10086000106A0F6A200E0E6E750E0D6E08C012F41F
:1008700007C011F4000129DC03C022F402C021F4F6
:1008800001C020F400C01FF410C026F40FC025F4EE
:100890000EC024F40DC023F434DC03C010F002C0F9
:1008A0000FF001C00EF000C00DF00401116B1151EA
:1008B000000127EC00F00401112B006E00509EA8EF
:1008C000FED7AD6E0C0E115DF2E1100EE96E08C0A0
:1008D00013F407C012F4000190DC2C0E9EA8FED782
:1008E000AD6E200E9EA8FED7AD6E890EE96E10C0CB
:1008F00015F40FC014F40EC013F40DC012F4060E5C
:100900000401166F000131DD2C0E9EA8FED7AD6EDE
:10091000200E9EA8FED7AD6E100EE96E0AC013F42D
:1009200009C012F46ADC0A0E9EA8FED7AD6E0D0E49
:100930009EA8FED7AD6EB36AB26AC282C2B2FED7BB
:10094000C3CF07F0C4CF08F0D8900B34026E0C343C
:10095000036E0250110FE96E000E0320EA6E08C00C
:10096000ECFFED5207C0EFFFB250B3CF03F0096EBA
:1009700003C00AF0106A0F6A200E0E6E770E0D6E1D
:1009800008C012F407C011F465EC00F003C022F4B3
:1009900002C021F401C020F400C01FF410C026F4EE
:1009A0000FC025F40EC024F40DC023F481EC00F038
:1009B00003C010F002C00FF001C00EF000C00DF037
:1009C0000401116B115100013DEC00F00401112BE9
:1009D000006E00509EA8FED7AD6E050E115DF2E1CF
:1009E000100EE96E08C013F407C012F4000105DC14
:1009F0002C0E9EA8FED7AD6E200E9EA8FED7AD6E23
:100A0000890EE96E10C015F40FC014F40EC013F473
:100A10000DC012F4060E0401166F0001A6DC2C0EA8
:100A20009EA8FED7AD6E200E9EA8FED7AD6E100E0E
:100A3000E96E0AC013F409C012F4FDEC00F0110EC7
:100A40000401126F125100013DEC00F00401122B61
:100A5000006E00509EA8FED7AD6E150E125DF2E13D
:100A60000B2AD8B40C2A0C50010802E20C6A0B6A5B
:100A7000040E116FFA0E126F000150EC00F0040129
:0A0A8000112FF8D70001A5D50300DF
:020000040030CA
:0E000000240E3F1E008381000FC00FE00F4052
:00000001FF
